:100000000C94A0000C94BE000C94BE000C94BE0096
:100010000C94BE000C94BE000C94BE000C94BE0068
:100020000C94BE000C94BE000C947B0A0C94BE0091
:100030000C94BE000C94BE000C94BE000C94BE0048
:100040000C94BE000C94BE000C94BE000C94BE0038
:100050000C94BF010C94BE000C94BE000C94610182
:100060000C94BE000C9425020C94BE000C94BE00AF
:100070000C94BE000C94DA000C94BE000C94BE00EC
:100080000C94BE000C94BE000C94BE000C94BE00F8
:100090000C94BE000C94BE000C94BE000C94BE00E8
:1000A0000C94BE000C94BE000C94BE001201000221
:1000B00002000020EB0318200010000000010902DC
:1000C0004300020100803209040000010202010025
:1000D000052400100105240103010424020605245F
:1000E000060001070583032000FF09040100020A3E
:1000F0000000000705810220000007050202200021
:10010000000C03410054004D0045004C0022034107
:1001100000560052002000550053004200200043CA
:1001200000440043002000440045004D004F000CF7
:100130000331002E0030002E0030000403090400BB
:1001400011241FBECFEFDAE0DEBFCDBF81E011E0AA
:10015000A0E0B1E0ECE5F0E202C005900D92A23221
:10016000B107D9F711E0A2E2B1E001C01D92AE3BA8
:10017000B107E1F70E94BD040C942C100C94000010
:1001800089ED86BD14BC84E085BD81E080936E005E
:10019000089581E480937C0010927B00EAE7F0E010
:1001A00080E8808380E980838EEC808383E3809382
:1001B0007E0008951F920F920FB60F9211248F9315
:1001C0009F9380913501882369F480917800909104
:1001D00079009093A3018093A20181E0809335017F
:1001E00081E447C080913501813069F480917800C5
:1001F000909179009093A5018093A40182E080936F
:10020000350184E436C080913501823069F48091F3
:100210007800909179009093A7018093A60183E0E4
:100220008093350185E425C080913501833091F4B8
:1002300080917800909179009093A9018093A80112
:1002400084E08093350187EC80937C0080E280938A
:100250007B0013C080913501843079F4809178005F
:10026000909179009093AB018093AA01109235018F
:1002700080E480937C0010927B008EEC80937A0067
:100280009F918F910F900FBE0F901F901895109215
:10029000850010928400E6E8F0E02FEF33E0318330
:1002A00020838FEF809380008AE0809381003183E8
:1002B000208310928200EFE6F0E0808181608083ED
:1002C00008951F920F920FB60F9211242F933F9310
:1002D0004F935F936F937F938F939F93AF93BF934E
:1002E000EF93FF9389ED86BD8091360190913701A0
:1002F0000196909337018093360180913801909157
:1003000039010196909339018093380180913A0127
:1003100090913B01019690933B0180933A0180912B
:100320003C0190913D01019690933D0180933C01E9
:1003300080913E0190913F01019690933F018093FF
:100340003E01809149018F5F80934901809149016D
:10035000823020F00E94470110924901FF91EF91F5
:10036000BF91AF919F918F917F916F915F914F91CD
:100370003F912F910F900FBE0F901F9018951F92D5
:100380000F920FB60F9211241092800010928100EC
:1003900010928500109284000F900FBE0F901F9056
:1003A0001895813049F48FEF93E0861B970B90935B
:1003B0008900809388000895823049F48FEF93E09C
:1003C000861B970B90938B0080938A00089583304F
:1003D00041F48FEF93E0861B970B90938D008093F1
:1003E0008C000895209133014091750190E030E038
:1003F000241B3109AC01429FC001439F900D529FC5
:10040000900D112464EB70E00E94970B9B0180918A
:100410007501280F311DC90108951F93182F862FCC
:100420000E94F201BC01812F0E94D1011F91089509
:1004300080538A3008F087500895809176018F5F4D
:10044000809376012B982F9808951F920F920FB6E4
:100450000F9211241F932F933F934F935F936F93AA
:100460007F938F939F93AF93BF93EF93FF932B9AB9
:100470008091B0018823E9F01091E90081E0809338
:10048000E90060E08091C80087FF08C0E62FF0E037
:100490008091CE00E65BFE4F80836F5F8091E80025
:1004A00085FFF0CF8AE491E00E94CB051093E9002C
:1004B00002C08091CE00FF91EF91BF91AF919F91CB
:1004C0008F917F916F915F914F913F912F911F91EC
:1004D0000F900FBE0F901F9018951F93682F80915B
:1004E000B001882379F01091E90081E08093E90060
:1004F0008091E80085FFFCCF8AE491E00E94CB0563
:100500001093E9001F9108958091B0018823D9F0DC
:100510008091C80085FF11C00E948205882369F080
:100520002F9A07C00E94A2058093790190E00E9453
:100530006F058091AC018823A9F780912401813057
:1005400011F4109224010895EF92FF920F93CF932C
:10055000DF9309B100950170499B0E5F4D9B0C5FC5
:10056000629B085F7F9B005F7E9B005E2091A201E3
:100570003091A3014091A4015091A5016091A60181
:100580007091A701E090A801F090A901C091AA0183
:10059000D091AB018DB79EB740970FB6F8949EBF30
:1005A0000FBE8DBFEDB7FEB731968AE491E0ADB7CF
:1005B000BEB712969C938E93119780E091E093833F
:1005C000828304831582378326835187408773870C
:1005D0006287F586E486D787C6870E942C0C8DB784
:1005E0009EB740960FB6F8949EBF0FBE8DBF88E1B0
:1005F00090E00E946D02DF91CF910F91FF90EF90FC
:10060000089580917A018C3409F499C08D3430F4C6
:100610008334B9F1843409F046C10AC0833509F442
:1006200044C0863509F43DC1823509F03CC160C043
:1006300090917B01892F90FF02C05C9A01C05C9869
:1006400081FF02C05E9A01C05E9882FF02C05F9A7D
:1006500001C05F9883FF02C02C9A01C02C9884FFD0
:1006600002C02D9A01C02D9885FF02C02E9A01C0AC
:100670002E9886FF02C0469A01C0469897FFC9C0CF
:1006800093C080917B0180FF02C02F9A01C02F98F8
:1006900081FF02C02B9A01C02B9882FF02C0299AC9
:1006A00001C0299883FF94C05EC080917B01803394
:1006B00009F45DC0813309F45EC0823309F45FC080
:1006C000833309F460C0843309F461C0853309F4CD
:1006D00062C0863309F463C0873309F465C084358A
:1006E000B1F18634C1F18934F1F18335C1F1DBC058
:1006F00080917B01803309F46FC0813309F470C0AD
:10070000823309F471C0833309F472C0843309F46D
:1007100073C0853309F474C0863309F475C0873318
:1007200009F477C0843509F447C0863409F448C019
:10073000893409F44DC0833509F446C0B4C08091B2
:100740007B018E3499F580917C01813011F42F9AD0
:10075000AAC0823011F42B9AA6C0833011F4299AD2
:10076000A2C0843011F42A9A9EC0853011F45C9A9C
:100770009AC0863011F45E9A96C0873011F45F9A61
:1007800092C0883011F42C9A8EC0893011F42D9AC1
:100790008AC08A3011F42E9A86C08B3011F4469AA2
:1007A00082C08C3009F07FC0479A7DC0863499F5AD
:1007B00080917C01813011F42F9875C0823011F442
:1007C0002B9871C0833011F429986DC0843011F4D6
:1007D0002A9869C0853011F45C9865C0863011F4A0
:1007E0005E9861C0873011F45F985DC0883011F465
:1007F0002C9859C0893011F42D9855C08A3011F4C5
:100800002E9851C08B3011F446984DC08C3009F0B1
:100810004AC0479848C0843509F045C090917C0192
:10082000913019F485B180582EC0923019F485B1F9
:1008300098E028C0933019F485B192E023C0943039
:1008400011F485B11FC0953019F48BB190E104C04B
:10085000963029F48BB190E489278BB924C0973066
:1008600019F48BB18058F9CF983019F485B190E123
:1008700009C0993019F485B190E204C09A3029F486
:1008800085B190E4892785B90EC09B3021F488B1E9
:1008900090E4892704C09C3031F488B1805888B92D
:1008A00002C00E94A4028DE080934A018AE08093F6
:1008B0004B018EE380934C0183E090E00E946D0237
:1008C0001092730108958AE090E7FC018491EBE0B7
:1008D000F0E73491ECE0F0E72491EDE0F0E794915B
:1008E0008C3231F4313121F42C3211F4923211F086
:1008F0000E94BD0408959FEF94B980EC87B980ED04
:100900008AB980E48DB910BA15B88FE388B98FE23F
:100910008BB98FEB8EB991BB0E9463041092480192
:10092000109247011092350185B7806885BF85B761
:10093000806885BF85B7806885BF85B7806885BFBB
:1009400085B7806885BF109273010E945A05E9EC53
:10095000F0E0808180688083E2EEF0E08081846056
:1009600080838091770183608093770181E096E0B6
:1009700062EA75E00E94E00B0895E7EDF0E0808107
:100980008160808388E08AB90E94200580E090E041
:10099000089513BE83B7856083BF8895089513BEFD
:1009A00083B7816083BF8895089513BE83B7836042
:1009B00083BF8895089513BE83B7876083BF8895EA
:1009C000089513BE83B78D6083BF8895089513BEC5
:1009D00083B78F6083BF889508958091C500846038
:1009E0008093C5008091C70080FFFCCF8091C50037
:1009F00081608093C5008091C500877F8093C5008A
:100A000008958091C50088608093C5008091C700DB
:100A100081FFFCCF8091C5008E7F8093C5008091BF
:100A2000C5008B7F8093C500089508950E948F0BA9
:100A30000E948402FBCF0E94920B0E947B040895C7
:100A40000E941B050E94160508958091BE01909199
:100A5000BF01A091C001B091C10185559A4AAA4A2F
:100A6000B54569F41092BE011092BF011092C00109
:100A70001092C101E0911901F0911A0109950895B0
:100A800085E59AEAAAEAB5E58093BE019093BF0195
:100A9000A093C001B093C101A895809160008061CE
:100AA0008093600088E080936000FFCF8091C80051
:100AB0008078089589E190E09093CD008093CC00F8
:100AC000E8ECF0E080818260808386E08093CA0059
:100AD000E9ECF0E080818861808381E00895282F2F
:100AE0008091C80085FFFCCF2093CE00822F08950F
:100AF0008091C80087FFFCCF8091CE0008951092AE
:100B0000AC0108958091AC018823B9F482E0809310
:100B1000E9008091E80082FF10C08091F20080938C
:100B2000AC01882351F48091E8008B7F8093E8002A
:100B30008091E8008F778093E8008091AC0181116B
:100B400081E0089582E08093E9008091AC018823E0
:100B500019F40E948205FBCF9091F1008091AC01C5
:100B600081508093AC01882351F48091E8008B7F01
:100B70008093E8008091E8008F778093E800892FC8
:100B800008958091E80090E025E0969587952A9554
:100B9000E1F781700895FC0181E08093E900262F40
:100BA00019C08091E80085FFFCCF04C0819180933B
:100BB000F10021508091E80085FF02C02223B1F7A7
:100BC0008091E8008E7F8093E8008091E8008F7725
:100BD0008093E800222329F7862F90E08F71907090
:100BE000892B71F48091E80085FFFCCF8091E800AB
:100BF0008E7F8093E8008091E8008F778093E800F3
:100C00000895DF93CF9300D0CDB7DEB79A83898361
:100C1000CE01019661E00E94CB0589819A810F90F7
:100C20000F90CF91DF910895E8EDF0E080818F770C
:100C300080838081806880838081806180838081DF
:100C400081608083789408958091D8008062809339
:100C5000D80082B7807F82BF82B78A6482BF82E079
:100C600089BD09B400FEFDCF8091D8008F7D8093AF
:100C7000D8008091E0008E7F8093E0008091E000BA
:100C8000877F8093E0008091E20081608093E200A2
:100C90008091E20088608093E20078940E94CE0602
:100CA000089580912201882371F48091D90080FFFA
:100CB0000AC08091D80080688093D80081E080933A
:100CC00022010E942406809131019091320190FF0F
:100CD00010C080913101909132019E7F909332013A
:100CE0008093310181E08093EA001092EA00109233
:100CF000B0011092E9008091E80083FF02C00E94D9
:100D00004A0808959091EB0091609093EB008093D6
:100D1000EC008091ED008270862B8093ED00809135
:100D2000ED0082608093ED008091EE00881F88279F
:100D3000881F08959091F40080E090FD06C08F5FB9
:100D4000873011F09695F9CF80E00895FB018093EC
:100D5000E90004C081918093F10041508091E80046
:100D600085FF02C04423B1F7842F0895FB018093CF
:100D7000E90004C08091F100819341508091E80026
:100D800085FF02C04423B1F7842F08958093E900C2
:100D9000EBEEF0E080818062808308951092E9009C
:100DA0008091EB0080FF02C080E008951092E9007E
:100DB00082E060E20E948206089580E008958091BA
:100DC000E800877F8093E800809140018093F100E4
:100DD000809141018093F100809142018093F10064
:100DE000809143018093F100809144018093F10050
:100DF000809145018093F100809146018093F1003C
:100E00008091E8008E7F8093E8008091E80080FF69
:100E1000FCCF8091E80082FFFCCF8091E8008B7FBF
:100E20008093E8008091E8008F778093E800089530
:100E30008091E800877F8093E8008091E80082FF3E
:100E4000FCCF8091F100809340018091F10080936C
:100E500041018091F100809342018091F1008093E3
:100E600043018091F100809344018091F1008093CF
:100E700045018091F100809346018091E8008B7FCD
:100E80008093E8008091E8008F778093E80080915C
:100E9000E8008E7F8093E8008091E80080FFFCCF1F
:100EA0002091400130914101409142015091430114
:100EB000569547953795279584E0220F331F441F99
:100EC000551F8A95D1F760E072E18AE790E00E94B1
:100ED000AA0B215030403093CD002093CC000895D0
:100EE0009091E800977F9093E8009091E8009E7FB2
:100EF0009093E800809374018091E80080FFFCCF1C
:100F00000895209177013091780180912501909189
:100F100026018217930711F480E00895309326018B
:100F20002093250183E08093E9008091E80085FD0E
:100F300002C081E0089581EA8093F10080E280930D
:100F4000F1001092F1001092F1001092F100109255
:100F5000F10082E08093F1001092F100809177011E
:100F60008093F100809178018093F1008091E800F6
:100F70008E7F8093E8008091E8008F778093E8006F
:100F800081E008958091E800877F8093E800809158
:100F9000E8008E7F8093E80081E0809324018091B7
:100FA000E80080FFFCCF0895DF93CF9300D0CDB74A
:100FB000DEB72091F1009091F1008132A9F42983EC
:100FC0009A83623239F0633251F06032A9F40E94A0
:100FD000180710C089819A810E9470070BC089810F
:100FE0009A810E94C20706C0813A31F4613221F42D
:100FF0000E94DF0681E001C080E00F900F90CF914A
:10100000DF910895FF920F931F9309EE10E083E0A4
:10101000F801808381EC60E20E94820681E0F801A1
:10102000808381E860E20E94820622E0F22EF801CD
:10103000F08280E860E20E948206EAEEF0E088E05A
:1010400080831082F082108284E0808310821F915E
:101050000F91FF90089509B400FC0BC082B7807F08
:1010600082BF82B78A6482BF82E089BD09B400FE74
:10107000FDCF8091D8008F7D8093D800809127018B
:10108000813039F48091E00082608093E00010921A
:1010900027010895DF93CF9300D0CDB7DEB78091BD
:1010A000E8008B7F8093E8009091F10090933001ED
:1010B0006091F1006630F9F0673068F4613009F44E
:1010C0001CC1613008F498C1633009F450C1653027
:1010D00009F0FDC1D6C0693009F4F5C06A3020F4CA
:1010E000683009F0F4C1B0C06A3009F4C1C16B3096
:1010F00009F0EDC1DBC1903809F0A3C010922801BE
:101100006091F1008091F100813019F0823089F412
:1011100006C082E18093B1018CEA90E005C083E4CF
:101120008093B1018EEB90E09093B3018093B20174
:1011300005C00E94DD06882309F4CEC18091F1002C
:101140008091F1008091F10089838091F1008A8380
:101150008091E800877F8093E80029813A8180911F
:10116000B10190E08217930758F48F719070892B2A
:1011700021F481E08093280105C01092280102C06B
:101180002093B1018091E8008F7E8093E800209148
:10119000B2013091B3014091B10122C08091E800C9
:1011A00084FF03C0F90190E00FC08091E80080FF48
:1011B000F5CFF8CF542F5150903249F09F5F849172
:1011C0008093F1003196452F9F01442399F7809138
:1011D000E80084FD12C08091E8008E7F8093E800D3
:1011E000442339F42093B2013093B3011092B1013A
:1011F0000AC08091E80084FFD8CF2093B2013093D9
:10120000B3014093B10180912801813069F480914C
:10121000E80084FD09C08091E80080FFFCCF809148
:10122000E8008E7F8093E8008091E80084FFFCCF87
:101230008091E8008F7E8093E8008091E8008B7FAA
:1012400053C1892F66E02FC19038C1F48091E80026
:10125000877F8093E8008091B0018093F1008091B6
:10126000E8008E7F8093E8008091E8008F7780937C
:10127000E8008091E80082FFFCCF0AC1892F68E076
:1012800012C19923E9F49091F1008091E3009F77D6
:101290008078982B9093E3008091E800877F80937B
:1012A000E8008091E8008E7F8093E8008091E8005C
:1012B00080FFFCCF8091E30080688093E30016C13B
:1012C000892F65E0F0C09923A9F49091F100923044
:1012D00008F002C18091E800877F8093E800909336
:1012E000B0018091E8008E7F8093E800892F0E94F2
:1012F0000208FCC0892F69E0D6C09330A8F5992375
:1013000009F441C0913009F4E7C08091F100909157
:10131000F100882309F0E0C0E091F100EF77E0935D
:10132000E9008091EB0080FF61C0EE23B1F0809175
:10133000EB0080618093EB0081E090E00E2E02C014
:10134000880F991F0A94E2F78093EA001092EA004E
:101350008091EB0088608093EB001092E900F0E050
:10136000E75DFE4F108239C0892F61E09CC0933049
:1013700008F03FC0913009F4AFC0913020F09230B6
:1013800009F0AAC003C08091F100A6C08091F100CD
:101390009091F100882309F09FC0E091F100EF7770
:1013A00051F48091EB0080628093EB008091E80023
:1013B000877F8093E800E093E9008091EB0080FF55
:1013C00015C08091EB0080628093EB001092E900E1
:1013D000F0E0E75DFE4F81E080838091E800877F49
:1013E0008093E8008091E8008E7F7EC01092E90033
:1013F00073C0892F63E057C0892F80588330A8F5C8
:101400008091F1008091F100E091F100913861F05C
:10141000923891F0903809F05FC08091E800877FA2
:101420008093E80081E013C08091E800877F80937B
:10143000E8001092F1000DC08091E800877F809352
:10144000E800F0E0EF77F070E75DFE4F8081809379
:10145000F1001092F1008091E8008E7F8093E80007
:101460008091E80082FFFCCF13C0892F60E01BC091
:101470009138B9F48091E800877F8093E8008091EB
:10148000E8008E7F8093E8008091E80082FFFCCF27
:101490008091E8008B7F8093E8008091E8008F774F
:1014A00023C0892F6AE00E94D40720C09130F1F454
:1014B0008091E800877F8093E8008091E8008E7F2C
:1014C0008093E8008091E80080FFFCCF0FC0892F57
:1014D0000E94D407882351F48091EB0080628093AE
:1014E000EB008091E800877F8093E8000F900F90D9
:1014F000CF91DF9108951F920F920FB60F92112492
:101500002F933F934F935F936F937F938F939F930B
:10151000AF93BF93EF93FF938091DA0080FF31C0C8
:101520008091D80080FF2DC08EEF8093DA008091EB
:10153000D90080FF19C081E08093220180913101A0
:1015400090913201826090933201809331018091B9
:10155000E20088608093E2000E9424068091E0000F
:101560008E7F8093E0000DC0109222011092B00196
:101570008091310190913201846090933201809387
:1015800031018091E10082FF09C08091E20082FF79
:1015900005C08BEF8093E1000E941D028091E10065
:1015A00080FF29C08091E20080FF25C081E0809308
:1015B00023018FEE8093E1008091310190913201FF
:1015C000806290933201809331018EEF8093E1002D
:1015D0008091E20080618093E2008091E2008F7D43
:1015E0008093E2008091D80080628093D80089B512
:1015F0008D7F89BD19BC8091E10084FF47C0809137
:10160000E20084FF43C009B400FC0BC082B7807FB6
:1016100082BF82B78A6482BF82E089BD09B400FEBE
:10162000FDCF8091D8008F7D8093D8009FEE90935E
:10163000E10080912301882349F18091E2008062DA
:101640008093E2008091E20088608093E2009093B2
:10165000E1008091E2008F7E8093E2008091310171
:101660009091320180649093320180933101809196
:10167000E20081608093E2008091E20080628093CA
:10168000E2008091E20088608093E2008091E100B6
:1016900085FF1CC08091E20085FF18C010922301D5
:1016A0008091E2008F7E8093E2008FED8093E100D5
:1016B0008091E2008F7D8093E200809131019091D2
:1016C0003201806890933201809331018091E10072
:1016D00083FF14C08091E20083FF10C01092AF011D
:1016E00087EF8093E1000E94CE06809131019091B6
:1016F000320191609093320180933101FF91EF911B
:10170000BF91AF919F918F917F916F915F914F9119
:101710003F912F910F900FBE0F901F9018950E9430
:10172000510608950E9414061092AF01089597FB88
:10173000092E07260AD077FD04D02ED006D000202F
:101740001AF4709561957F4F0895F6F790958195FD
:101750009F4F0895A1E21A2EAA1BBB1BFD010DC0CD
:10176000AA1FBB1FEE1FFF1FA217B307E407F50751
:1017700020F0A21BB30BE40BF50B661F771F881F2D
:10178000991F1A9469F760957095809590959B01C3
:10179000AC01BD01CF010895AA1BBB1B51E107C0DD
:1017A000AA1FBB1FA617B70710F0A61BB70B881FF1
:1017B000991F5A95A9F780959095BC01CD01089580
:1017C0000F931F93CF93DF938C01EB01009731F4BC
:1017D0006115710519F420E030E038C081E090E037
:1017E0006EE070E00E942D0EFC019C01009771F1EB
:1017F00080E88383209771F0D387C28781E8838351
:101800008091B4019091B501892B21F4F093B50139
:10181000E093B40101151105C9F011870087838198
:10182000826083838091B6019091B701892B71F416
:10183000F093B701E093B6018091B8019091B9019E
:10184000892B21F4F093B901E093B801C901DF912C
:10185000CF911F910F910895AEE0B0E0E2E3FCE07C
:101860000C9403100D891E8986E08C831A830983EA
:101870008FEF9FE79E838D839E01275E3F4FCE01B2
:1018800001966F89788DA9010E94500C2F813885AF
:10189000020F131FF80110822E96E4E00C941F1023
:1018A000ABE0B0E0E6E5FCE00C94F50F3C012B0169
:1018B0005A01FC0117821682838181FD03C06FEFFC
:1018C0007FEFC6C19AE0892E1E010894211C311CAD
:1018D000F3012381F20123FD859123FF81912F01E3
:1018E000882309F4B2C1853239F423FD859123FFA1
:1018F00081912F01853229F490E0B3010E946B0F92
:10190000E7CF982FFF24EE249924FFE1FF15D0F0B4
:101910009B3269F09C3228F4903259F0933291F462
:101920000EC09D3249F0903369F441E024C052E08A
:10193000F52A84E0F82A28C098E0F92A25C0E0E1D9
:10194000FE2A22C0F7FC29C0892F80538A3070F408
:10195000F6FE05C0989C902C1124980E15C0E89CAA
:10196000E02C1124E80EF0E2FF2A0EC09E3229F48A
:10197000F6FC6BC140E4F42A07C09C3619F450E829
:10198000F52A02C0983649F4F20123FD959123FF10
:1019900091912F01992309F0B8CF892F8554833075
:1019A00018F08052833038F444E050E0A40EB51EA5
:1019B0005FE359830FC0933631F0933779F0933555
:1019C00009F056C020C0F5018081898342E050E0D3
:1019D000A40EB51E610101E010E012C0F501C08047
:1019E000D180F6FC03C06FEF7FEF02C0692D70E07D
:1019F00042E050E0A40EB51EC6010E94600F8C01AB
:101A00005FE7F52214C0F501C080D180F6FC03C069
:101A10006FEF7FEF02C0692D70E042E050E0A40E4E
:101A2000B51EC6010E944E0F8C0150E8F52AF3FE48
:101A300007C01AC080E290E0B3010E946B0FEA94E5
:101A40008E2D90E008171907A8F30EC0F601F7FCD9
:101A50008591F7FE81916F0190E0B3010E946B0FB9
:101A6000E110EA94015010400115110579F7EAC020
:101A7000943611F0993669F5F7FE08C0F50120811A
:101A800031814281538184E090E00AC0F501808178
:101A900091819C01442737FD4095542F82E090E0CE
:101AA000A80EB91E9FE6F92257FF09C05095409530
:101AB000309521953F4F4F4F5F4FE0E8FE2ACA0116
:101AC000B901A1012AE030E00E94970FD82ED21868
:101AD00040C0953729F41F2D1F7E2AE030E01DC03D
:101AE0001F2D197F9F3661F0903720F4983509F04B
:101AF000ACC00FC0903739F0983709F0A6C004C0C9
:101B000028E030E00AC0106114FD146020E130E0EC
:101B100004C014FD166020E132E017FF08C0F50193
:101B2000608171818281938144E050E008C0F501B9
:101B300080819181BC0180E090E042E050E0A40E01
:101B4000B51EA1010E94970FD82ED2188FE7F82E4C
:101B5000F122F6FE0BC05EEFF522D91438F4F4FE44
:101B600007C0F2FC05C08FEEF82202C01D2D01C097
:101B7000192DF4FE0DC0FE01ED0DF11D80818033A5
:101B800019F499EEF92208C01F5FF2FE05C003C0E8
:101B90008F2D867809F01F5F0F2DF3FC14C0F0FE27
:101BA0000FC01E1510F09D2C0BC09D2C9E0C911A81
:101BB0001E2D06C080E290E0B3010E946B0F1F5FF4
:101BC0001E15C0F304C01E1510F4E11A01C0EE2466
:101BD00004FF0FC080E390E0B3010E946B0F02FF8F
:101BE0001DC001FD03C088E790E00EC088E590E0CD
:101BF0000BC0802F867891F001FF02C08BE201C0FC
:101C000080E2F7FC8DE290E0B3010E946B0F06C00A
:101C100080E390E0B3010E946B0F9A94D914C0F353
:101C2000DA94F101ED0DF11D808190E0B3010E9485
:101C30006B0FDD20A9F706C080E290E0B3010E949F
:101C40006B0FEA94EE20C1F743CEF30166817781F2
:101C5000CB012B96E2E10C9411100F931F93CF93BD
:101C6000DF93689F8001699F100D789F100D1124EC
:101C7000C8010E94490EEC01009729F060E070E075
:101C8000A8010E94590FCE01DF91CF911F910F91B2
:101C90000895CF93DF93BC018230910510F462E088
:101CA00070E0A091BC01B091BD01ED01E0E0F0E079
:101CB00040E050E021C0888199818617970769F438
:101CC0008A819B81309719F09383828304C090931B
:101CD000BD018093BC01FE0134C06817790738F458
:101CE0004115510519F08417950708F4AC01FE0160
:101CF0008A819B819C01E9012097E9F641155105F4
:101D0000A9F1CA01861B970B049708F4BA01E0E019
:101D1000F0E02AC08D919C91119784179507F9F4F2
:101D20006417750781F412968D919C9113973097E3
:101D300019F09383828304C09093BD018093BC010A
:101D4000FD0132964FC0CA01861B970BFD01E80FBB
:101D5000F91F6193719302978D939C9343C0FD018A
:101D6000828193819C01D9011097A1F68091BA01DB
:101D70009091BB01892B41F480911D0190911E012E
:101D80009093BB018093BA0140911F0150912001B3
:101D90004115510541F44DB75EB780911B019091FB
:101DA0001C01481B590B2091BA013091BB0124172B
:101DB0003507B0F4CA01821B930B8617970780F092
:101DC000AB014E5F5F4F8417950750F0420F531FD2
:101DD0005093BB014093BA01F9016193719302C022
:101DE000E0E0F0E0CF01DF91CF910895CF93DF9352
:101DF000009709F450C0EC0122971B821A82A0912F
:101E0000BC01B091BD01109709F140E050E0AC1762
:101E1000BD0708F1BB83AA83FE0121913191E20F36
:101E2000F31FAE17BF0779F48D919C911197280F7E
:101E3000391F2E5F3F4F3983288312968D919C91D5
:101E400013979B838A834115510571F4D093BD018B
:101E5000C093BC0120C012968D919C911397AD0147
:101E6000009711F0DC01D3CFFA01D383C283219113
:101E70003191E20FF31FCE17DF0769F48881998152
:101E8000280F391F2E5F3F4FFA01318320838A814B
:101E90009B8193838283DF91CF910895FC0105900C
:101EA000615070400110D8F7809590958E0F9F1F5C
:101EB0000895DC0101C06D9341505040E0F7089552
:101EC000FC016150704001900110D8F78095909509
:101ED0008E0F9F1F08950F931F93CF93DF938C0155
:101EE000EB018B8181FF1BC082FF0DC02E813F81E2
:101EF0008C819D812817390764F4E881F981019369
:101F0000F983E88306C0E885F985802F0995892B38
:101F100031F48E819F8101969F838E8302C00FEFE3
:101F20001FEFC801DF91CF911F910F910895FA0122
:101F3000AA27283051F1203181F1E8946F936E7F08
:101F40006E5F7F4F8F4F9F4FAF4FB1E03ED0B4E0F9
:101F50003CD0670F781F891F9A1FA11D680F791F3A
:101F60008A1F911DA11D6A0F711D811D911DA11D4B
:101F700020D009F468943F912AE0269F112430195B
:101F8000305D3193DEF6CF010895462F4770405DF6
:101F90004193B3E00FD0C9F7F6CF462F4F70405DA5
:101FA0004A3318F0495D31FD4052419302D0A9F700
:101FB000EACFB4E0A6959795879577956795BA95FA
:101FC000C9F700976105710508959B01AC010A2EC0
:101FD00006945795479537952795BA95C9F7620F97
:101FE000731F841F951FA01D08952F923F924F923B
:101FF0005F926F927F928F929F92AF92BF92CF9299
:10200000DF92EF92FF920F931F93CF93DF93CDB7A1
:10201000DEB7CA1BDB0B0FB6F894DEBF0FBECDBF19
:1020200009942A88398848885F846E847D848C84EA
:102030009B84AA84B984C884DF80EE80FD800C81F3
:102040001B81AA81B981CE0FD11D0FB6F894DEBFD6
:0C2050000FBECDBFED010895F894FFCF46
:10205C00432533642C2534642C2534642C253464BA
:10206C002C2534642C2533640000382000C2010078
:02207C00000062
:00000001FF
